:203D000012010002FFFFFF40B50420010001010203010A0600020000004001000902890088
:203D200001010080370904000001FF000000070586020002000904000101FF00010007050C
:203D400082010014010904000201FF00010007058201000C010904000301FF000100070502
:203D600082010004010904000401FF000100070582010004020904000501FF0001000705F5
:203D800082010004030904000601FF000100070582010004040904000701FF0001000705CD
:053DA000820100020495
:203DA6000902390002010080370904000001FF000000070586024000000904000101FF0010
:193DC600010007058201FF03010904000201FF00010007058201000201AF
:203DE000040309040E0373006900670072006F006B0010036600780032006C0061006600B9
:203E0000770022035300610069006E0053006D006100720074002000440044005300310048
:063E20003200300000003A
:040000000201B9320E
:01000B0032C2
:0100130032BA
:01001B0032B2
:0100230032AA
:03002B000203AD20
:030033000202E4E2
:01003B003292
:01004300328A
:01004B003282
:01005300327A
:01005B003272
:01006300326A
:03006B000202E7A7
:03007300020D2A51
:03007B000208EA8E
:03008300020395E0
:03008B000202FF6F
:0300930002034A1B
:03009B000208E771
:0300A300020D54F7
:0300AB00020D55EE
:0300B300020D56E5
:0300BB00020D59DA
:0300C300020D2902
:0300CB00020D46DD
:0300D300020D47D4
:0300DB00020D49CA
:0300E3000208EC24
:0300EB00020DD132
:0300F3000208E818
:0300FB000208E90F
:030103000208EB04
:03010B000208EDFA
:030113000208EEF1
:03011B00020DB41E
:03012300020D5278
:03012B00020D576B
:03013300020D5A60
:03013B00020D5C56
:03014300020D5357
:03014B00020D584A
:03015300020D5B3F
:03015B00020D5D35
:03016300020DB3D7
:03016B00020D4A38
:03017300020D4C2E
:03017B00020D4E24
:03018300020D501A
:03018B00020D4B17
:03019300020D4D0D
:03019B00020D4F03
:0301A300020D51F9
:0301AB00020D48FA
:0301B300020D2812
:0C021200750800E4F509F50AC200C201FD
:030230000201B612
:0301B6000207D865
:20023300E582FF70407E0EE4FDFC7401B51302801C7402B5130280197405B513028016742B
:200253000AB5130280137414B5131680107B0280647B0680607B00805C7B0480587B0880BB
:200273005475820022BF01497E307D027401B51302801C7402B51302801B7405B51302804F
:200293001A740AB5130280197414B5132080187B007C0280207B107C02801A7B007C008095
:2002B300147B107C00800E7B207C0080087582002275820022EEF4FFE5A05207EE5B4FF565
:2002D300A0EDF4FFE5B15207ED5C4FF5B175820122C2DC32C0E0C082C083D2005391EF901A
:2002F300E65D7401F0D083D082D0E032C021C0E0C0F0C082C083C007C006C005C004C0032D
:20031300C002C001C000C0D075D000758200120C185391EF90E65D7410F0D0D0D000D0012A
:20033300D002D003D004D005D006D007D083D082D0F0D0E0D02132C021C0E0C0F0C082C044
:2003530083C007C006C005C004C003C002C001C000C0D075D000758201120C185391EF9085
:20037300E65D7420F0D0D0D000D001D002D003D004D005D006D007D083D082D0F0D0E0D082
:200393002132C0E0C082C083D2015391EF90E65D7408F0D083D082D0E032C0E0C007C00639
:2003B300C0D075D000AEB17F006306048EB1E509450A6010150974FFB50902150AE509457B
:2003D3000A700100C2CFD0D0D006D007D0E032E582FF30E00BADB17E004305088DB1800361
:2003F30053B1F7EF30E408AEB14306018EB12253B1FE22AF82BF01028003BF021174072FC4
:20041300FF90E618F090E61AEFF0758201227582002290E6F574FFF000000090E60474806E
:20043300F000000090E6047482F000000090E6047486F000000090E604E4F02290E6F574A6
:20045300FFF0000000E50870057E06FF80047E027F0090E648EEF022D2871204257EE87FFB
:2004730003EE24FFFCEF34FFFD8C068D07EC4D70F0E5BB30E7FB00000090E6D07428F000F7
:20049300000090E6D1E4F0E50870057E06FF80047E047F008EBB00E4F509F50A22AF8290B7
:2004B300E680E030E7067D1C7E3D80047DA67E3D8F03E4CBC4CB6BCB54F0CB6BFC74162BDF
:2004D300FBE43CFCEB2DFDEC3EFC7E80EFF508703590E612E4F090E61474E0F090E6E27432
:2004F30001F08D828C838EF0120DB590E625F074012DFAE43CFB8E078A828B838FF0120DF9
:20051300B590E624F02290E61274D8F090E614E4F090E6D204F08D828C838EF0120DB59009
:20053300E621F00DBD00010C8D828C838EF0120DB5FF90E62074075FF08D828C838EF0125D
:200553000DB5C423541F90E64004F022AF827E00EE75F007A4FCADF024D6F582ED340DF5C6
:2005730083E493FBB5070280080EBE11E375820022EC24D6FCED340DFD74062CF582E43D09
:20059300F583E49390E601F075AF07759DE4759E008C828D83A3E49390E67CF08C828D8386
:2005B300A3A3E49390E67CF07401F0E4F0F0F0F0F08C828D83A3A3A39390E67CF08C828D79
:2005D30083A3A3A3A3E49390E67CF07401F0E4F0F0F0F0F08C828D83A3A3A3A3A39390E651
:2005F3007CF07444F0F0E4F0F0F0F0F0F0F0F0F0F0F0F0F07F0090E67CE4F00FBF6000401D
:20061300F575820122AF82BF00028049BF01028062BF02028067BF050302069ABF0A030278
:2006330006A4BF14030206AEBF69028014BF6A028019BF6E02801EBF78028023BF9666800B
:200653002875CAF075CBD87582012275CA7375CBDF7582012275CA7875CBEC7582012275A1
:20067300CA3C75CBF67582012275CA1875CBFC7582012275CA0C75CBFE7582012275CA067C
:2006930075CBFF7582012275CA9C75CBFF7582012275CACE75CBFF7582012275CAE775CBEE
:2006B300FF7582012275820022AD13AE14AF158D828E838FF0E508120D2B75820122E58258
:2006D3007006850B821204B0758201227582002275820122AF82C00712044FD007007509BA
:2006F300E8750A03BFE0004015EF2419401090E68AE4F090E68BF090E6A0E020E1F9BFE0B9
:2007130000500302078EEF2419500302078EEF2420FE2E90072A73800C800A801B8026805C
:2007330033803E8049EF2420FF90E740E0F5138F821202337582012290E740E0F582120584
:200753005F7582012290E740E0FFBF010312046B7582012290E740E0F582120406758201F7
:200773002290E740E0F5821203E27582012290E740E0F58212061875820122758200229024
:20079300E613E4F090E615F0D28790E6C2E4F090E6C37480F090E6C0E4F090E6F4F0120402
:2007B3004F75130175820012023375130175820112023375820112055F7582021204067550
:2007D30082000204B090E600E053E0E7F0120792E500D2E890E668E0FF43070890E668EF48
:2007F300F090E65CE0FF43070190E65CEFF0E0FF43071090E65CEFF0E0FF43072090E65C44
:20081300EFF0E0FF43070890E65CEFF0D2DDD2AF75CA0C75CBFE75C800D2ADD2CA90E680FD
:20083300E043E00AF09005DC120D5E90E680E053E0F7F090E672E4F090E671F090E670F061
:2008530075B6FF75B4FF75B2FF10000280031208EF10010280F390E682E043E0C0F090E6C8
:20087300817401F0AE877F004306018E8700000000000000E50E701C90E682E030E6079068
:20089300E682E020E0D090E682E030E70790E682E020E1C290E682E030E60790E682E020AF
:2008B300E00E90E682E030E7A090E682E030E199900005120D5E90E680E0FF43070190E67E
:1408D30080EFF090000F120D5E90E680E053E0FEF002085C39
:200DD600308000030000EA1E8000030000AA180100020140EA100101020040EA0F0100027F
:200DF6000140AA0C0201020040EA0B0101020040AA080302020040EA060202020040AA058A
:200E16000302020040AA040605020040EA030504020040AA020C0B020040EA011817020021
:170E360040EA32302F020040EA147877020040EA0AF0EF020040EA7A
:0108E70032DE
:0108E80032DD
:0108E90032DC
:0108EA0032DB
:0108EB0032DA
:0108EC0032D9
:0108ED0032D8
:0108EE0032D7
:0601E800E478FFF6D8FDEB
:12021E00750D00750E00750FA675103D75111C75123D77
:2008EF0090E6B9E0FF24F45003020A13EF240A83F582EF241083F583E473213D13591313D5
:20090F0075137B92B4EE09090A090A0A090A09090909120A95E5826003020A2F90E6A0E075
:20092F00FF7E0043070190E6A0EFF0020A2F120B29E5826003020A2F90E6A0E0FF7E0043AF
:20094F00070190E6A0EFF0020A2F120B77E5826003020A2F90E6A0E0FF7E0043070190E683
:20096F00A0EFF0020A2F120C43020A2F1206DFAF8290E740EFF090E68AE4F090E68B04F08B
:20098F00020A2F90E6BAE0F5821206E3E5826003020A2F90E6A0E0FF7E0043070190E6A0B2
:2009AF00EFF0020A2F90E6BCE0FF75130C7514007515408F821206BCE582701190E6A0E053
:2009CF00FF7E0043070190E6A0EFF0805390E740E50CF090E68AE4F090E68B04F0804190C6
:2009EF00E6BCE0FF90E6BAE0F50B8F821206D1E582702D90E6A0E0FF7E0043070190E6A085
:200A0F00EFF0801C90E6B9E0F5821206E7E582700F90E6A0E0FF7E0043070190E6A0EFF02E
:200A2F0090E6A0E0FF43078090E6A0EFF022AF82747F5FFE24F75003020A91EE240A83F5B1
:200A4F0082EE240D83F583E4736A6E8191859189918D0A0A0A0A0A0A0A0A0A90E6A022EF6C
:200A6F0030E7067EA27FE680047EA17FE68E828F832290E6A32290E6A42290E6A52290E64F
:200A8F00A6229000002290E6B8E0FFBF80028022BF81028008BF82028037020B2190E74034
:200AAF00E4F090E741F090E68AF090E68B7402F08064E50E25E0FFE50D420790E740EFF0A8
:200ACF0090E741E4F090E68AF090E68B7402F0804590E6BCE0F582120A3DAE82AF838E0489
:200AEF008F05EE4F7003F582228C828D83E0FC30E0067E017F0080047E007F0090E740EED6
:200B0F00F090E741E4F090E68AF090E68B7402F08004758200227582012290E6B8E0FF60CF
:200B2F0005BF0237801190E6BAE0FFBF0105750E0080317582002290E6BAE0701A90E6BC2B
:200B4F00E0F582120A3DAE82AF83E0FD5305FE8E828F83EDF0800D7582002290E6B9E0F598
:200B6F00820206E77582012290E6B8E0FF6008BF02028020020C0B90E6BAE0FFBF02030215
:200B8F000C1490E6BAE0FFBF0106750E01020C147582002290E6BAE0705E90E6BCE0F5822B
:200BAF00120A3DAE82AF83EE4F7003F582228E828F83E0FD7C004305018E828F83EDF090CF
:200BCF00E6BCE0FF53070F90E6BCE0FE530680E4C423CEC423541F6ECE541FCE6ECE30E473
:200BEF000244E0FD90E683EE2FF0E0FF7E0043072090E683EFF0800D7582002290E6B9E069
:200C0F00F5820206E775820122AF827E0110AF027E00EF600E750F1C75103D7511A67512E4
:200C2F003D800C750FA675103D75111C75123DEE1392AF2290E6BBE0FFBF01028019BF02FA
:200C4F00028024BF0302802CBF0603020CFDBF0703020D0D020D1A7E007F3D90E6B3EFF04C
:200C6F0090E6B47400F02290E6B3E510F090E6B4E50FF0227DE07E3D7F8090E6BAE0F51348
:200C8F007B008B020BEAB5130280428D008E018F028D828E838FF0120DB528F8E439F988DE
:200CAF000589068A0774012DF9E43EFA8F0489828A838CF0120DB5F9B9030280067D007E16
:200CCF00007F00ED4E6006C3E5139B50B5ED4E600F8D038E0490E6B3ECF090E6B4EDF02290
:200CEF0090E6A0E0FF43070190E6A0EFF0227E127F3D90E6B3EFF090E6B47412F02290E602
:190D0F00B3E512F090E6B4E511F02290E6A0E0FF43070190E6A0EFF022A8
:2001C6007900E94400601B7A00900E4D780075923CE493F2A308B800020592D9F4DAF27565
:0201E60092FF86
:010D28003298
:010D29003297
:010D2A003296
:1B0D2B0020F71130F6138883A88220F509F6A8837583002280FEF280F5F022C7
:010D4600327A
:010D47003279
:010D48003278
:010D49003277
:03004300023F0079
:203F00000202E700020D2A000208EA00020395000202FF0002034A000208E700020D53004A
:203F2000020D5400020D5500020D5600020D5900020D2900020D4600020D4700020D4900B2
:203F40000208EC00020D5300020DD1000208E8000208E9000208EB000208ED000208EE0060
:203F6000020DB400020D5300020D5300020D5300020D5200020D5700020D5A00020D5C00BD
:203F8000020D5800020D5B00020D5D00020DB300020D4A00020D4C00020D4E00020D5000B2
:183FA000020D4B00020D4D00020D4F00020D5100020D4800020D280007
:010D4A003276
:010D4B003275
:2001EE007800E84400600A790075923CE4F309D8FC7800E84400600C7900903C00E4F0A3A7
:04020E00D8FCD9FA45
:010D4C003274
:010D4D003273
:010D4E003272
:010D4F003271
:010D50003270
:010D5100326F
:010D5200326E
:010D5300326D
:010D5400326C
:010D5500326B
:010D5600326A
:010D57003269
:010D58003268
:010D59003267
:010D5A003266
:010D5B003265
:010D5C003264
:010D5D003263
:200D5E00AE82AF8390E600E05418C423541F70057CB1FD801C90E600E05418C423541FFBA5
:200D7E00BB01067A617B0180047AC27B028A048B058C138D14151374FFB513021514E5131B
:150D9E00451470F1EE24FFFAEF34FFFB8A068B07EA4B70DD2298
:010DB300320D
:010DB400320C
:0D01B900758121120DD2E58260030201B6AE
:1C0DB50020F71430F6148883A88220F507E6A88375830022E280F7E49322E0224D
:010DD10032EF
:040DD2007582002204
:00000001FF
